:020000020000FC
:0200000006C038
:020004001EC01C
:10000C003BC00FE90DBF0FE007BB00E008BB02E0EF
:10001C000FBD02E003BF0FEF06BF04E009BF00E213
:10002C000BBF00E105BB00E305BF00E808B966277C
:10003C0078948895FECF26B324FF07C072B70027AB
:10004C0002BF703498F021D011C002B7083088F08C
:10005C00112712BF003820F0EE24FF24662706C0BB
:10006C00EE0CFF1C6395003208F0E39400E205BF30
:10007C001895070F02BFFACF08D08395883220F06D
:10008C008827332700E305BF1895603120F0CE1484
:10009C00DF0419F405D0EE24FF24670166270895C8
:1000AC003030E1F50E2D06950A34C1F587010E7F2F
:1000BC00102702951027012F169516950127102F42
:1000CC001695012701701E2D1170101739F50F2D83
:1000DC001F2D12951095011709F54F2D4F7008B370
:1000EC00413039F0423051F0443069F0483081F001
:1000FC0015C000FDC09800FFC09A0FC001FDC1984B
:10010C0001FFC19A0AC002FDC29802FFC29A05C043
:0E011C0003FDC39803FFC39A00C031E00895AD
:00000001FF
